:020000040000FA
:040000008FEF00F08E
:020008009ED088
:08001800ECD00C6E960E046E94
:10002000980E056E55D8D8B4CA90D8A4CA80FC0FD3
:10003000D8A0CA92D8B0CA82800E046E960E056E01
:10004000980E086E096ACAB025D8CAB223D842D819
:100050000404CB6E04C006F005C007F000500A6E21
:100060000B6E003C0B6A4BD809500C2E0AD0BE6EAA
:100070000C0EBD6E08BEBD8A08BCBD889394CA84B0
:100080001200BB6E0C0EBA6E08BEBA8A08BCBA88E3
:100090009492F5D700D8D890083205320432120075
:1000A000076A066EFF0E0626072200D0D8A01200AF
:1000B000030E056EE70E02D8F5D7056AFE0F046E33
:1000C000E86A055AD8A012000000040600D0F8D74C
:1000D000096A086A100EF36E0534083609360650B0
:1000E000085C0750095805E30650085E0750095A96
:1000F000D88004360536F32EEFD704501200065090
:100100000A02F3CF08F0F4CF09F007500A02F350C7
:10011000092606500B02F350092608501200F86A0F
:100120004F0EAF6E240EAC6E900EAB6E0001C69AF1
:10013000470E926EE00E936EC00E946E070EB46E74
:100140000F0EC16EA1D09EAA1BD0060EAB1412E1F9
:10015000E1CF36F0E2CF37F0382A1EEE80F038508B
:10016000E126000EE222AECFE7FF36C0E1FF37C046
:10017000E2FF1100AE50AE50AB98AB8811000AD030
:10018000F2A408D0F294114A122A817A106AD6CFCA
:100190000FF0110011003850395C14E0392AE9CF12
:1001A00004F0EACF05F00EEE80F03950E926000E9B
:1001B000EA22EF50046E04C0E9FF05C0EAFFD880D0
:1001C000120004D0E868046ED8A012001200386A49
:1001D000396A9D8A9F8AF28EF28C12009D9A0EEEE9
:1001E00080F0000EEE6AE82EFDD7386A396A9D8AE3
:1001F0001200F29ED8CF5AFEE8CF5BFEE0CF5CFE45
:10020000E9CF5DFEEACF5EFEE1CF5FFEE2CF60FEAA
:10021000D9CF61FEDACF62FEF6CF63FEF7CF64FE80
:10022000F5CF65FEF3CF66FEF4CF67FEA6CF68FE7E
:10023000F28E0001A192D40EB26EB30EB36EF29E96
:100240005ACED8FF5BCEE8FF5CCEE0FF5DCEE9FF83
:100250005ECEEAFF5FCEE1FF60CEE2FF61CED9FF66
:1002600062CEDAFF63CEF6FF64CEF7FF65CEF5FF10
:1002700066CEF3FF67CEF4FF68CEA6FFF28E1000C5
:100280009EA8FED7AD6E1200949A8B9A94988B9884
:1002900093908A9093928A9294968B9694908B9056
:1002A000939A8A9A2C6A306A006A280E066E260E85
:1002B000076E020EB2DE006A280E066E260E076E6C
:1002C000010EABDE316A939A8A8A320EE9DE939A86
:1002D0008A9A2A6A356A7BDF81DFCD6AF294F28AD4
:1002E000870ED56EB16AA192A082B26AB36AD08E2F
:1002F000A292B10EB16E4FDF136EBB0E135C05E31D
:10030000FE0E135C01E2156A9CD113AE19D0156A7A
:100310008A0E135C05E113C015F0166817680FD03C
:100320009A0E135C05E113C015F01868196807D020
:10033000BA0E135C04E113C015F01C681D6881D16E
:10034000155202E17ED17DD18A0E155CD8A488D0E9
:10035000162803E113C016F081D013C017F0270E42
:10036000165CD8A051D0580E165CD8B04DD0006A9B
:10037000280E066E260E076E020E4FDE30523BE14F
:10038000175209E12EC000F0280E066E260E076EE9
:10039000010E43DE09D0D8901734006E280E066E89
:1003A000260E076E010E39DE2B80D6CF0FF0D7CF89
:1003B00010F02DC002F0016AD890023601C046F05C
:1003C00002C047F046C001F047C002F001500F24C0
:1003D000226E02501020236E000E1120246E000E9B
:1003E0001220256E24C054F025C055F022C062F0C2
:1003F00023C063F008D02B90006A280E066E260EEC
:10040000076E010E0ADE29D0780E165C04E13590E5
:100410002A908B9A22D0790E165C04E135922A92AA
:100420008B981BD07A0E165C04E135942A948A903E
:1004300014D07B0E165C04E135962A968A920DD074
:100440007C0E165C04E135982A988B9606D07D0EBA
:10045000165C03E1359A2A9A8B901668F2D0F1D097
:100460009A0E155CD8A4D3D0182803E113C018F055
:10047000CCD013C019F01952D8A477D0270E185C2D
:10048000D8A048D0580E185CD8B044D0006A280EC6
:10049000066E260E076E020E0DEC00F0305230E1B3
:1004A0002EC000F0280E066E260E076E010E0DEC13
:1004B00000F02B80D6CF0FF0D7CF10F02DC002F078
:1004C000016AD890023601C046F002C047F046C02B
:1004D00001F047C002F001500F24226E025010209C
:1004E000236E000E1120246E000E1220256E24C0F3
:1004F00054F025C055F022C062F023C063F009D04B
:100500002B90006A280E066E260E076E010E0DEC6B
:1005100000F029D0780E185C04E135902A908B9A6F
:1005200022D0790E185C04E135922A928B981BD068
:100530007A0E185C04E135942A948A9014D07B0ECC
:10054000185C04E135962A968A920DD07C0E185CD0
:1005500004E135982A988B9606D07D0E185C03E14D
:10056000359A2A9A8B9018686CD0270E185C17E37E
:10057000580E185C14E2006A280E066E260E076EEE
:10058000010E0DEC00F02B90D8901934006E280E5F
:10059000066E260E076E020E0DEC00F035D0780EBA
:1005A000185C32E37F0E195C06E218C01AF019C01D
:1005B0001BF01ED929D0780E185C04E135802A90F2
:1005C0008B8A22D0790E185C04E135822A928B88BE
:1005D0001BD07A0E185C04E135842A948A8014D0EA
:1005E0007B0E185C04E135862A968A820DD07C0E3B
:1005F000185C04E135882A988B8606D07D0E185C3D
:1006000003E1358A2A9A8B8018681BD01AD0AA0E6B
:10061000155C0AE11A2803E113C01AF003D013C0D5
:100620001BF0E6D80ED00DD0BA0E155C0AE11C28DE
:1006300003E113C01CF004D013C01DF03DEC05F025
:1006400000D02A52D8B4AED02AA01BD048C024F083
:1006500049C025F056C022F057C023F0D6CF0FF086
:10066000D7CF10F022500F5C23501058245011584F
:100670002550125812502518D8B0800AD8B8ABECC3
:1006800005F02AA21BD04AC024F04BC025F058C068
:1006900022F059C023F0D6CF0FF0D7CF10F0225060
:1006A0000F5C2350105824501158255012581250E6
:1006B0002518D8B0800AD8B8CEEC05F02AA41BD0F3
:1006C0004CC024F04DC025F05AC022F05BC023F08E
:1006D000D6CF0FF0D7CF10F022500F5C2350105818
:1006E000245011582550125812502518D8B0800A9D
:1006F000D8B8F1EC05F02AA61BD04EC024F04FC0AC
:1007000025F05CC022F05DC023F0D6CF0FF0D7CF2C
:1007100010F022500F5C23501058245011582550CF
:10072000125812502518D8B0800AD8B814EC06F028
:100730002AA81BD050C024F051C025F05EC022F082
:100740005FC023F0D6CF0FF0D7CF10F022500F5C50
:100750002350105824501158255012581250251863
:10076000D8B0800AD8B837EC06F02AAA1BD052C0FD
:1007700024F053C025F060C022F061C023F0D6CF32
:100780000FF0D7CF10F022500F5C23501058245098
:1007900011582550125812502518D8B0800AD8B8D0
:1007A0005AEC06F02BA022D054C024F055C025F0FE
:1007B00062C022F063C023F0D6CF0FF0D7CF10F085
:1007C00022500F5C235010582450115825501258B5
:1007D00012502518D8B0800A09E7006A280E066E64
:1007E000260E076E010E0DEC00F02B907BEF01F052
:1007F000780E1A5C32E135A02DD02A80D6CF0FF0CA
:10080000D7CF10F01B1C036E7F0E03140D6E0E6A03
:100810000DC002F0016AD890023601C03AF002C061
:100820003BF03AC001F03BC002F001500F24226EB1
:1008300002501020236E000E1120246E000E122094
:10084000256E24C048F025C049F022C056F023C0D0
:1008500057F002D02A908B9A08D1790E1A5C32E1B7
:1008600035A22DD02A82D6CF0FF0D7CF10F01B1C87
:10087000036E7F0E03140D6E0E6A0DC002F0016A46
:10088000D890023601C03CF002C03DF03CC001F0FF
:100890003DC002F001500F24226E02501020236E42
:1008A000000E1120246E000E1220256E24C04AF086
:1008B00025C04BF022C058F023C059F002D02A9234
:1008C0008B98D3D07A0E1A5C32E135A42DD02A84CD
:1008D000D6CF0FF0D7CF10F01B1C036E7F0E031482
:1008E0000D6E0E6A0DC002F0016AD890023601C08A
:1008F0003EF002C03FF03EC001F03FC002F00150A8
:100900000F24226E02501020236E000E1120246E40
:10091000000E1220256E24C04CF025C04DF022C0E0
:100920005AF023C05BF002D02A948A909ED07B0EAE
:100930001A5C32E135A62DD02A86D6CF0FF0D7CF5C
:1009400010F01B1C036E7F0E03140D6E0E6A0DC09B
:1009500002F0016AD890023601C040F002C041F0B6
:1009600040C001F041C002F001500F24226E02503D
:100970001020236E000E1120246E000E1220256E12
:1009800024C04EF025C04FF022C05CF023C05DF0C3
:1009900002D02A968A9269D07C0E1A5C32E135A880
:1009A0002DD02A88D6CF0FF0D7CF10F01B1C036EA6
:1009B0007F0E03140D6E0E6A0DC002F0016AD8900E
:1009C000023601C042F002C043F042C001F043C011
:1009D00002F001500F24226E02501020236E000EF0
:1009E0001120246E000E1220256E24C050F025C068
:1009F00051F022C05EF023C05FF002D02A988B969F
:100A000034D07D0E1A5C31E135AA2DD02A8AD6CF9A
:100A10000FF0D7CF10F01B1C036E7F0E03140D6E6A
:100A20000E6A0DC002F0016AD890023601C044F08F
:100A300002C045F044C001F045C002F001500F244F
:100A4000226E02501020236E000E1120246E000E24
:100A50001220256E24C052F025C053F022C060F051
:100A600023C061F002D02A9A8B901A6812001E6887
:100A70001200206812001F681200210E1C5C0AE19F
:100A80001DC02CF0D8902C342E6E2F6A2F362E4A93
:100A90002F2A26D0220E1C5C03E11DC02DF020D091
:100AA000400E1C5C0FE11DC030F0305203E02E6A96
:100AB0002F6A07D0D8902C342E6E2F6A2F362E4AEC
:100AC0002F2A0ED0420E1C5C07E11D5203E131902B
:100AD00024D801D0318004D07B0E1C5CD8B402D85D
:100AE0001C6812002A6A2B6A8B9A8B988A908A92C9
:100AF0008B968B90939A8A9A356A006A280E066EB6
:100B0000260E076E020E0DEC00F0006A280E066E2F
:100B1000260E076E010E0DEF00F02A6A2B6A8B9AE3
:100B20008B988A908A928B968B90939A8A9A356A40
:100B3000006A280E066E260E076E020E0DEC00F0FF
:100B4000006A280E066E260E076E010E0DEC00F0F0
:100B50002C6A316A120035B003D02A908B9A1DD0CE
:100B6000D6CF0FF0D7CF10F03AC001F03BC002F063
:100B700001500F24226E02501020236E000E11200F
:100B8000246E000E1220256E24C048F025C049F0C6
:100B900022C056F023C057F0827A120035B203D03B
:100BA0002A928B981DD0D6CF0FF0D7CF10F03CC033
:100BB00001F03DC002F001500F24226E02501020BF
:100BC000236E000E1120246E000E1220256E24C00C
:100BD0004AF025C04BF022C058F023C059F082786B
:100BE000120035B403D02A948A901DD0D6CF0FF0CE
:100BF000D7CF10F03EC001F03FC002F001500F24EB
:100C0000226E02501020236E000E1120246E000E62
:100C10001220256E24C04CF025C04DF022C05AF0A1
:100C200023C05BF08170120035B603D02A968A92F9
:100C30001DD0D6CF0FF0D7CF10F040C001F041C08B
:100C400002F001500F24226E02501020236E000E7D
:100C50001120246E000E1220256E24C04EF025C0F7
:100C60004FF022C05CF023C05DF08172120035B8F5
:100C700003D02A988B961DD0D6CF0FF0D7CF10F087
:100C800042C001F043C002F001500F24226E025016
:100C90001020236E000E1120246E000E1220256EEF
:100CA00024C050F025C051F022C05EF023C05FF098
:100CB0008276120035BA03D02A9A8B901DD0D6CFF7
:100CC0000FF0D7CF10F044C001F045C002F0015042
:100CD0000F24226E02501020236E000E1120246E6D
:100CE000000E1220256E24C052F025C053F022C001
:0C0CF00060F023C061F082701200FFD79A
:020000040030CA
:0300010006170ED1
:020005008580F4
:060008000FC00FE00F40E5
:00000001FF
